:050000007581407590C0
:0200060075B0D3
:200009001201791200DDAC091200901200A812018B2000031200472000EE12002B20B4E82A
:2000290080E4C0E0E509B4600280090509E5092400D4F509FC1200781200C4D0E022C0E066
:20004900E509B4000280131509E509540FB40F00E509400424109410F509FC120000120006
:20006900C4D0E022C2B5120184B2B2120184227B5A1200901200A812018BDBF8227F0DB7AF
:050089009FCDDBFB0F21
:20008F00DFC0E0ECC4540F90008693F50CEC540F90008693F50CD0E022850B90C2B712009F
:2000AF00BDD2B7850C90C2901200BDD29022750D00D50DFD22120140750AA01200F3750AAC
:2000CF00001200F385090A1200F312014F22120140750AA01200F3750A001200F312012AB3
:2000EF00850A0922C0E0E50A7D083392B4120167DDF8D2B4120167D2B312016720B400C2C6
:20010F00B3D0E022C0E0E47D083167D2B33167A2B433C2B3DDF3F50AD0E022120140750A1C
:20012F00A11200F312011312014F22D2B412015C22D2B4D2B3120167C2B4120167C2B3223D
:20014F00C2B4120167D2B3120167D2B422120167D2B3120167C2B3227E030000DEFC227FED
:20016F000A7EE60000DEFCDFF8227F647EE60000DEFCDFF8227D64316EDDFC22C0E0C0003A
:20018F00758910758AB0758CB0D2B5750E00750F00D28CE4B50902C2B53088FD050EA80E5D
:1901AF00B805F6750E00050FE50F2400D4F50FB470E2C28CD000D0E02207
:00000001FF
